:020000040000FA
:100000000C947F000C94A7000C94A7000C94A700FC
:100010000C94A7000C94A7000C94A7000C94A700C4
:100020000C94A7000C94A7000C94A7000C94A700B4
:100030000C94A7000C94A7000C94A7000C94A700A4
:100040000C94F8040C94A7000C94C6040C94A0041F
:100050000C94A7000C94A7000C94A7000C94A70084
:100060000C94A7000C94A70050000000000024008E
:1000700027002A00486F6D65536572766572494F97
:100080004578742076007D002C2248223A007B229D
:1000900054223A004552523A20444854206661693D
:1000A0006C656420746F207265616400000000005C
:1000B000250028002B0000000008000201000003BA
:1000C0000407000000000000000000000000230002
:1000D00026002900040404040404040402020202A9
:1000E00002020303030303030102040810204080FB
:1000F0000102040810200102040810204205112406
:100100001FBECFEFD8E0DEBFCDBF11E0A0E0B1E071
:10011000E2EBF4E102C005900D92A832B107D9F7E5
:1001200021E0A8E2B1E001C01D92AD3FB207E1F7C6
:1001300010E0CFE7D0E004C02197FE010E94510AF1
:10014000CE37D107C9F70E948F050C94570A0C943B
:100150000000CF92DF92EF92FF92CF93DF93B091A6
:10016000F101A0E08111AB2F8091F20190E0880FA6
:10017000991FAC0146535F4FC090F701D090F80132
:10018000E090F901F090FA0130E020E0FA01C59129
:10019000D491E881B90190E080E0EB23EA130AC032
:1001A0002F5F3F4F6C157D058E059F0578F36FEF30
:1001B0007FEFCB01DF91CF91FF90EF90DF90CF9059
:1001C0000895AF92BF92CF92DF92EF92FF920F937A
:1001D0001F93CF93DF936C017B018B01040F151FDD
:1001E000EB015E01AE18BF08C017D10759F0699145
:1001F000D601ED91FC910190F081E02DC6010995A9
:10020000892B79F7C501DF91CF911F910F91FF9055
:10021000EF90DF90CF90BF90AF900895FC01538D89
:10022000448D252F30E0842F90E0821B930B5417D0
:1002300010F0CF96089501970895FC01918D828D5D
:10024000981761F0A28DAE0FBF2FB11D5D968C91F6
:10025000928D9F5F9F73928F90E008958FEF9FEF35
:100260000895FC01918D828D981731F0828DE80FF1
:10027000F11D858D90E008958FEF9FEF0895FC01AB
:10028000918D228D892F90E0805C9F4F821B910978
:100290008F73992708958DE491E00E943F0121E03A
:1002A000892B09F420E0822F089580E090E0892BCB
:1002B00029F00E944B0181110C9400000895FC016B
:1002C000A48DA80FB92FB11DA35ABF4F2C91848DB7
:1002D00090E001968F739927848FA689B7892C9314
:1002E000A089B1898C91837080648C93938D848D67
:1002F000981306C00288F389E02D80818F7D80836A
:100300000895EF92FF920F931F93CF93DF93EC0129
:1003100081E0888F9B8D8C8D98131AC0E889F989AC
:10032000808185FF15C09FB7F894EE89FF896083AF
:10033000E889F98980818370806480839FBF81E030
:1003400090E0DF91CF911F910F91FF90EF90089572
:10035000F62E0B8D10E00F5F1F4F0F731127E02E4D
:100360008C8D8E110CC00FB607FCFACFE889F98985
:10037000808185FFF5CFCE010E945F01F1CFEB8D2B
:10038000EC0FFD2FF11DE35AFF4FF0829FB7F89459
:100390000B8FEA89FB8980818062CFCF0F931F93F7
:1003A000CF93DF938C01D0E0C0E0F801EC0FFD1F8C
:1003B0006491662341F08DE491E00E948101892BD4
:1003C00011F02196F2CFCE01DF91CF911F910F91C5
:1003D0000895CF93DF93EC01888D8823B9F0AA8923
:1003E000BB89E889F9898C9185FD03C0808186FDF0
:1003F0000DC00FB607FCF7CF8C9185FFF2CF80813F
:1004000085FFEDCFCE010E945F01E9CFDF91CF9153
:100410000895833081F028F4813099F08230A9F07A
:1004200008958730A9F08830C9F08430B1F4809104
:1004300080008F7D03C0809180008F778093800043
:10044000089584B58F7784BD089584B58F7DFBCFE3
:100450008091B0008F778093B00008958091B000B4
:100460008F7DF9CFCF93DF93282F30E0F901EA5445
:10047000FF4F8491F901E851FF4FD491F901EC52FB
:10048000FF4FC491CC23A1F081110E940902EC2FEF
:10049000F0E0EE0FFF1FE653FF4FA591B491EC91F2
:1004A000ED2381E090E009F480E0DF91CF910895A1
:1004B00080E090E0FACFCF93DF9390E0FC01E85129
:1004C000FF4F24918C529F4FFC0184918823D1F0DF
:1004D00090E0880F991FFC01E659FF4FA591B49158
:1004E000FC01E455FF4FC591D491623071F49FB780
:1004F000F8943C91822F809583238C93E8812E2B56
:1005000028839FBFDF91CF9108958FB7F894EC9126
:100510002E2B2C938FBFF6CF3FB7F89480912D01EF
:1005200090912E01A0912F01B091300126B5A89B8A
:1005300005C02F3F19F00196A11DB11D3FBFBA2F75
:10054000A92F982F8827BC01CD01620F711D811D35
:10055000911D42E0660F771F881F991F4A95D1F7BA
:1005600008958F929F92AF92BF92CF92DF92EF92B7
:10057000FF924B015C010E948C026B017C010E9486
:100580008C026C197D098E099F09683E73408105B4
:100590009105A8F321E0821A9108A108B10888EE1C
:1005A000C80E83E0D81EE11CF11C81149104A10443
:1005B000B10429F7FF90EF90DF90CF90BF90AF90FC
:1005C0009F908F9008952FB7F894609129017091B2
:1005D0002A0180912B0190912C012FBF08958F92B9
:1005E0009F92AF92BF92CF92DF92EF92FF920F93C2
:1005F0001F93CF93DF93CDB7DEB7C054D1400FB672
:10060000F894DEBF0FBECDBF0E94E3020091F3015C
:100610001091F4012091F5013091F6016B017C01FC
:10062000C01AD10AE20AF30A97018601003D174079
:1006300021053105B0F48091FB01C05CDE4F0FB69F
:10064000F894DEBF0FBECDBFDF91CF911F910F9108
:10065000FF90EF90DF90CF90BF90AF909F908F90E2
:1006600008956093F3017093F4018093F5019093E2
:10067000F6011092EE011092ED011092EC01109231
:10068000EB011092EA0162E08091EF010E945B02AF
:1006900061E070E080E090E00E94B10261E0809152
:1006A000EF010E945B022091EF0130E0F901EA5472
:1006B000FF4F8491F901E851FF4F0491F901EC5289
:1006C000FF4F1491112391F081110E940902E12F33
:1006D000F0E0EE0FFF1FE455FF4FA591B4918FB7E7
:1006E000F894EC9100950E230C938FBF8091F0014C
:1006F0008551823020F58BE291E10197F1F762E0BC
:100700008091EF010E945B028091FC0190E08230B9
:10071000910538F0880F991F880F991F0597019749
:10072000F1F7F89480E00E94A9006F3F7F4F8F4F50
:100730009F4F61F41092FB01789480E07ECF64E1DA
:1007400070E080E090E00E94B102D9CF81E00E9489
:10075000A9006F3F7F4F8F4F9F4F61F3CE010196EE
:100760007C015E019FEBA91A9EEFB90A870180E028
:100770000E94A900F801608371838283938381E0E2
:100780000E94A900F8016483758386839783085FBC
:100790001F4FA016B10659F7789430E020E0F7011A
:1007A00080809180A280B380448155816681778169
:1007B000FFEF8F169F06AF06BF0631F04F3F8FEF5A
:1007C00058076807780719F41092FB01B6CFF901B2
:1007D00083E0F595E7958A95E1F7E651FE4F808134
:1007E000880F84169506A606B70618F180832F5F3A
:1007F0003F4F98E0E90EF11C2832310581F6409117
:10080000EE012091EA018091EB01280F3327331F7D
:100810008091EC01280F311D8091ED01820F932F03
:10082000911D99274817190679F681E08093FB01FD
:1008300004CF8160DBCFFC0101900020E9F7319704
:10084000AF01481B590BBC018DE491E00C94E10011
:100850008F929F92AF92BF920F931F93CF93DF938C
:10086000CDB7DEB7A1970FB6F894DEBF0FBECDBFF0
:1008700019A2423008F44AE08E010F5D1F4F842E0A
:10088000912CB12CA12CA50194010E942F0AE62FD6
:10089000B901CA01EA30F4F4E05DD801EE938D01AC
:1008A000232B242B252B79F790E080E0109719F06B
:1008B000CD010E941B04A1960FB6F894DEBF0FBEB7
:1008C000CDBFDF91CF911F910F91BF90AF909F90BF
:1008D0008F900895E95CE1CFCF93DF930E941B04D2
:1008E000EC0182E191E00E941B048C0F9D1FDF91BF
:1008F000CF910895CF93C82F88E690E00E94CE0153
:100900006C2F70E090E080E04AE00E94280485E1CE
:1009100091E00E941B04EC2FF0E0E15DFE4F80812E
:10092000882359F087E191E00E946C0465E070E053
:1009300080E090E0CF910C94B10289E191E0F4CF96
:100940001F920F920FB60F9211242F933F934F9344
:100950005F936F937F938F939F93AF93BF93EF9327
:10096000FF938DE491E00E945F01FF91EF91BF91B1
:10097000AF919F918F917F916F915F914F913F9137
:100980002F910F900FBE0F901F9018951F920F92EE
:100990000FB60F9211242F938F939F93EF93FF9392
:1009A000E0915D01F0915E018081E0916301F09141
:1009B000640182FD1BC09081809166018F5F8F73FF
:1009C00020916701821741F0E0916601F0E0E35B5E
:1009D000FE4F958F80936601FF91EF919F918F91CC
:1009E0002F910F900FBE0F901F9018958081F4CF1C
:1009F0001F920F920FB60F9211242F933F938F9354
:100A00009F93AF93BF938091290190912A01A09168
:100A10002B01B0912C013091280123E0230F2D37B9
:100A200058F50196A11DB11D20932801809329013D
:100A300090932A01A0932B01B0932C0180912D015A
:100A400090912E01A0912F01B09130010196A11D2E
:100A5000B11D80932D0190932E01A0932F01B0938F
:100A60003001BF91AF919F918F913F912F910F9046
:100A70000FBE0F901F90189526E8230F0296A11D18
:100A8000B11DD2CFEDE4F1E01382128288EE93E043
:100A9000A0E0B0E084839583A683B78384E091E0EF
:100AA0009183808385EC90E09587848784EC90E047
:100AB0009787868780EC90E0918B808B81EC90E02B
:100AC000938B828B82EC90E0958B848B86EC90E00C
:100AD000978B868B118E128E138E148EAAEEB1E038
:100AE00081E115968C93159786E116968C9316974F
:100AF000E9EFF0E0E4911796EC931797E5EEF0E05C
:100B0000E4911896EC93189740E85EE360E070E09B
:100B10001D964D935D936D937C93509708957894B3
:100B200084B5826084BD84B5816084BD85B58260F2
:100B300085BD85B5816085BD80916E0081608093A3
:100B40006E0010928100809181008260809381000C
:100B5000809181008160809381008091800081601C
:100B6000809380008091B10084608093B100809177
:100B7000B00081608093B00080917A00846080939F
:100B80007A0080917A00826080937A0080917A0066
:100B9000816080937A0080917A00806880937A00E7
:100BA0001092C100E0915D01F0915E0182E08083CE
:100BB000E0915901F0915A011082E0915B01F091AE
:100BC0005C0180E1808310926501E0916101F09108
:100BD000620186E08083E0915F01F0916001808195
:100BE00080618083E0915F01F09160018081886085
:100BF0008083E0915F01F091600180818068808353
:100C0000E0915F01F091600180818F7D808384E7B6
:100C100090E00E94CE018BE191E00E946C04C2E062
:100C200062E08C2F0E945B02CF5FC630C9F701E300
:100C300011E0C2E08C2F0E94320221E0892B09F4DE
:100C400020E0F80121938F01CF5FC63099F762E071
:100C50008091EF010E945B020E94E302605D774099
:100C6000810991096093F3017093F4018093F50178
:100C70009093F60187E38093FC01C0E0D0E035E477
:100C8000A32E31E0B32E45E3E42E41E0F42E51E3F0
:100C9000C52E51E0D52E12E0812F0E94320201E0D4
:100CA000892B09F400E0F50181915F01081751F0EB
:100CB0000E94E302F7016083718382839383F501CD
:100CC00031970083F60180810817E1F00E94E3026A
:100CD000F70140805180628073806419750986092C
:100CE00097096B3F71058105910560F0F60100835E
:100CF0000E94E302F7016083718382839383812FD3
:100D00000E947A041F5FFFEFCF1ADF0A24E0E20E91
:100D1000F11C163009F60E94E3020091490110917E
:100D20004A0120914B0130914C01601B710B820BE9
:100D3000930B61367A4E8105910508F4C9C00E9473
:100D4000E3026093490170934A0180934B019093B1
:100D50004C0182E00E947A0483E00E947A0484E0DD
:100D60000E947A0485E00E947A040E94EF028823A0
:100D700049F08091F0018B3028F08D3050F0855192
:100D80008230C8F1812C912C20ECA22E2FE7B22EBC
:100D90001EC06091EB0170E090E080E00E940809C5
:100DA0002DEC3CEC4CEC5DE30E94BD096B017C0139
:100DB0006091EA0170E090E080E00E9408099B01E8
:100DC000AC01C701B6010E945F084B015C010E94A3
:100DD000EF02882309F474C08091F0018C3009F48B
:100DE00082C0D8F48B3091F1C12CD12C80ECE82E4C
:100DF0008FE7F82E55C06091EA017091EB017627DC
:100E00006727762790E080E00E9406092DEC3CECF5
:100E10004CEC5DE30E94BD09D8CF8551823020F7AC
:100E20001091EC01612F70E0762F662766277F779F
:100E30008091ED01682B90E080E00E9406092DEC86
:100E40003CEC4CEC5DE30E94BD0969C06091EC0193
:100E500070E090E080E00E9406096B017C01109137
:100E6000ED0117FF0AC0AC019B0160E070E080E873
:100E70009FEB0E945E086B017C011F70612F70E088
:100E800090E080E00E9408092DEC3CEC4CEC5DE326
:100E90000E94BD09A70196010E945F086B017C01B9
:100EA000A5019401C501B4010E942A0A811108C05C
:100EB000A7019601C701B6010E942A0A8823C1F141
:100EC00084E990E00E94CE0182E191E00E941B043F
:100ED000209709F4D4CE0E944B01882309F4CFCE89
:100EE0000E940000CCCE1091EC01612F70E090E0E8
:100EF00080E00E9406096B017C016091ED016F703A
:100F000070E090E080E00E9408092DEC3CEC4CEC95
:100F10005DE30E94BD09A70196010E945F086B0175
:100F20007C0117FFBDCFF7FAF094F7F8F094B8CF33
:100F30008EE890E00E94CE0126013701E89477F810
:100F40002FEF3FEF4FE75FE7C301B2010E942A0A8C
:100F500081113DC02FEF3FEF4FE75FE7C301B201C3
:100F60000E94CB0818169CF58FE191E00E941B04AB
:100F700088E890E00E94CE01C501B4010E94D0082B
:100F80006B01770FEE08FF084AE0C701B601F7FED4
:100F90000DC06DE28DE491E00E9481016627772704
:100FA000CB016C197D098E099F094AE00E94280433
:100FB00086E890E00E94CE0182E191E00E941B044D
:100FC00065E070E080E090E00E94B10281CF2FEFF9
:100FD0003FEF4FE75FE4C701B6010E94B80918165A
:100FE0001CF483E291E0C2CF2FEF3FEF4FE75FECBD
:100FF000C701B6010E94CB0887FDF3CF20E030E0A7
:10100000A901C701B6010E94CB0887FF09C06DE2A4
:101010008DE491E00E948101F7FAF094F7F8F094E2
:101020002AE037ED43EA5BE3C701B6010E945F089F
:101030002B013C010E94D7086B017C010E9406092C
:101040009B01AC01C301B2010E945E082B013C016F
:101050004AE0C701B6010E9428046EE28DE491E0E7
:101060000E94810120E030E040E251E4C301B2017E
:101070000E94BD092B013C010E94D7086B01F12C95
:10108000E12C4AE0C701B6010E942804C701B6015D
:101090000E9406099B01AC01C301B2010E945E08D7
:1010A00020E030E040E251E40E94BD090E94D708F0
:1010B00090E080E04AE00E9428045ACF5058BB27B5
:1010C000AA270E9476080C947E090E94700938F0C5
:1010D0000E94770920F039F49F3F19F426F40C940C
:1010E0006D090EF4E095E7FB0C946709E92F0E9467
:1010F0008F0958F3BA17620773078407950720F022
:1011000079F4A6F50C94B1090EF4E0950B2EBA2FE4
:10111000A02D0B01B90190010C01CA01A0011124FD
:10112000FF27591B99F0593F50F4503E68F11A16A9
:10113000F040A22F232F342F4427585FF3CF46953A
:1011400037952795A795F0405395C9F77EF41F165C
:10115000BA0B620B730B840BBAF09150A1F0FF0F26
:10116000BB1F661F771F881FC2F70EC0BA0F621F12
:10117000731F841F48F4879577956795B795F79502
:101180009E3F08F0B0CF9395880F08F09927EE0F97
:101190009795879508950E94430908F481E0089582
:1011A0000E94D7086894B1110C94B20908950E9466
:1011B000970988F09F5798F0B92F9927B751B0F049
:1011C000E1F0660F771F881F991F1AF0BA95C9F7CB
:1011D00014C0B13091F00E94B109B1E008950C94AF
:1011E000B109672F782F8827B85F39F0B93FCCF362
:1011F000869577956795B395D9F73EF49095809548
:10120000709561957F4F8F4F9F4F0895E89409C067
:1012100097FB3EF490958095709561957F4F8F4F29
:101220009F4F9923A9F0F92F96E9BB279395F6953F
:10123000879577956795B795F111F8CFFAF4BB0FBD
:1012400011F460FF1BC06F5F7F4F8F4F9F4F16C021
:10125000882311F096E911C0772321F09EE8872FAB
:10126000762F05C0662371F096E8862F70E060E067
:101270002AF09A95660F771F881FDAF7880F9695E0
:10128000879597F90895990F0008550FAA0BE0E884
:10129000FEEF16161706E807F907C0F01216130638
:1012A000E407F50798F0621B730B840B950B39F478
:1012B0000A2661F0232B242B252B21F408950A26DE
:1012C00009F4A140A6958FEF811D811D089597F91E
:1012D0009F6780E870E060E008959FEF80EC0895DC
:1012E00000240A9416161706180609060895002405
:1012F0000A9412161306140605060895092E03947F
:10130000000C11F4882352F0BB0F40F4BF2B11F4F2
:1013100060FF04C06F5F7F4F8F4F9F4F089557FD51
:101320009058440F551F59F05F3F71F04795880F53
:1013300097FB991F61F09F3F79F0879508951216EA
:1013400013061406551FF2CF4695F1DF08C0161696
:1013500017061806991FF1CF869571056105089447
:101360000895E894BB2766277727CB0197F908955E
:101370000E94430908F48FEF08950E94D0090C944D
:101380007E090E94700938F00E94770920F09523A9
:1013900011F00C9467090C946D0911240C94B20996
:1013A0000E948F0970F3959FC1F3950F50E0551F70
:1013B000629FF001729FBB27F00DB11D639FAA27AA
:1013C000F00DB11DAA1F649F6627B00DA11D661FF9
:1013D000829F2227B00DA11D621F739FB00DA11D1A
:1013E000621F839FA00D611D221F749F3327A00DD4
:1013F000611D231F849F600D211D822F762F6A2F70
:1014000011249F5750409AF0F1F088234AF0EE0FD4
:10141000FF1FBB1F661F771F881F91505040A9F701
:101420009E3F510580F00C9467090C94B2095F3F10
:10143000E4F3983ED4F3869577956795B795F7953D
:10144000E7959F5FC1F7FE2B880F911D96958795B5
:1014500097F908950E944309880B990B0895A1E21A
:101460001A2EAA1BBB1BFD010DC0AA1FBB1FEE1F1E
:10147000FF1FA217B307E407F50720F0A21BB30B69
:10148000E40BF50B661F771F881F991F1A9469F7E5
:1014900060957095809590959B01AC01BD01CF0141
:1014A0000895EE0FFF1F0590F491E02D0994F89434
:1014B000FFCF000000008101E1000E01E9013F01C2
:1014C0001D0131010D0A003D0048004C00302E3155
:0A14D00000696E66006F766600008A
:107E0000112484B714BE81FFF0D085E080938100F7
:107E100082E08093C00088E18093C10086E0809377
:107E2000C20080E18093C4008EE0C9D0259A86E02C
:107E300020E33CEF91E0309385002093840096BBD3
:107E4000B09BFECF1D9AA8958150A9F7CC24DD24C4
:107E500088248394B5E0AB2EA1E19A2EF3E0BF2EE7
:107E6000A2D0813461F49FD0082FAFD0023811F036
:107E7000013811F484E001C083E08DD089C08234E0
:107E800011F484E103C0853419F485E0A6D080C0E4
:107E9000853579F488D0E82EFF2485D0082F10E0AE
:107EA000102F00270E291F29000F111F8ED06801E7
:107EB0006FC0863521F484E090D080E0DECF843638
:107EC00009F040C070D06FD0082F6DD080E0C81688
:107ED00080E7D80618F4F601B7BEE895C0E0D1E017
:107EE00062D089930C17E1F7F0E0CF16F0E7DF06D8
:107EF00018F0F601B7BEE89568D007B600FCFDCFD4
:107F0000A601A0E0B1E02C9130E011968C91119780
:107F100090E0982F8827822B932B1296FA010C0160
:107F200087BEE89511244E5F5F4FF1E0A038BF0790
:107F300051F7F601A7BEE89507B600FCFDCF97BE46
:107F4000E89526C08437B1F42ED02DD0F82E2BD052
:107F50003CD0F601EF2C8F010F5F1F4F84911BD097
:107F6000EA94F801C1F70894C11CD11CFA94CF0C13
:107F7000D11C0EC0853739F428D08EE10CD085E9AC
:107F80000AD08FE07ACF813511F488E018D01DD067
:107F900080E101D065CF982F8091C00085FFFCCF94
:107FA0009093C60008958091C00087FFFCCF809118
:107FB000C00084FD01C0A8958091C6000895E0E648
:107FC000F0E098E1908380830895EDDF803219F02E
:107FD00088E0F5DFFFCF84E1DECF1F93182FE3DFCA
:107FE0001150E9F7F2DF1F91089580E0E8DFEE27F6
:047FF000FF270994CA
:027FFE00040479
:00000001FF
